:020000020000FC
:1000000002C080C087C0F8940FED0DBF55D08FEFB0
:1000100078940BB10078E9F38F3F89F4ACB00A2DE6
:10002000003F49F00F70B02E0A2D02950F70C02EC0
:100030000CE0C01610F48A2DECCF8FEFEACFACB0F5
:10004000803F11F10A2D0031E8F4C0E6D0E0CC0C7D
:10005000CC0CCC0CCC0DD81D0B2D0170D02EB69431
:10006000CB0DD81D00E0D01631F40881007FA02A06
:10007000A8828FEFCECF08810F70A294A02AA88209
:100080008FEFC7CF8FEFC5CF08E0A01610F08FEF2E
:10009000C0CF5A2DC0E6D0E0F2E0E4EA00E65030EE
:1000A00021F0E00FF81D5A95FACF30E6059109933B
:1000B0003A95E1F78FEFADCF02EF01BB0FEF07BB32
:1000C000C09A00E0802E10E020E0B0E0A0EC02E159
:1000D0002D930A95E9F720E0B0E0A0E600E62D9325
:1000E0000A95E9F700E00AB90BB906E003B900E0A8
:1000F00002B90AE009B900E10AB90EE005BF00EC57
:100100000BBF08950F930FB70F9310E00F910FBF20
:100110000F9118950F930FB70F933F93CF93DF93E2
:10012000EF93FF93012F13950C5138F0003C28F406
:10013000602F6695017051F03BC0FF91EF91DF9108
:10014000CF913F910F910FBF0F911895562E569456
:1001500056945694462F4770A0E6B0E0782C652C54
:100160008894661C771C661C771C661C771CA60D81
:10017000B71DC1ECD0E030E07C91032F017011F08D
:100180007295A3957F70F2E0E4E2782C672E889454
:10019000661C771C661C771C661C771C640E781C1A
:1001A000E60DF71D949099923395303129F7C5CF1C
:1001B00032E33A953030E9F70000A0ECB0E0A395C7
:1001C0002D9128BB2695000000000000000028BBF0
:1001D0002695000000000000000028BB26950000C6
:1001E00000000000000028BB269500000000000071
:1001F000000028BB2695000000000000000028BB7E
:100200002695000000000000000028BB2695000095
:1002100000000000000028BB2D91A23D91F60000D7
:10022000C0988BCF0000000000000000FFFFFFFF20
:10023000FFFFFFFFFF818181818181FF7EFFFFFF43
:10024000FFFFFF7E0000183C3C1800000000001873
:100250001800000000001824241800000008087F7F
:100260001C1422007F7F7F00F7F7F7007700DD0086
:100270007700DD00007E7E7E7E7E7E000808080816
:1002800008080808FFFF7E3C3C7EFFFF427E42429A
:10029000427E42420000000024DB000000000049D2
:1002A000B600000000000000000000000000000098
:1002B000000000000000000000000000000000003E
:1002C000000000000000000000000000000000002E
:1002D000000000000000000000000000000000001E
:1002E000000000000000000000000000000000000E
:1002F00000000000000000000000000000000000FE
:1003000000000000000000000000000000000000ED
:100310000000000000000000050000000050000088
:10032000000000007000000000000000000000005D
:100330000050000700000005000000000000000061
:100340000000000000070000700000000000050031
:100350000000500000000000000000001111111109
:100360001111111100000000000000001111110115
:100370001111111151545555551554155151110163
:10038000111015155151010000001515515501119D
:100390001010551511510010101011155155011163
:1003A0001010551551510100000015155151110142
:1003B000111015155154555555155415111111019C
:1003C000111111110000000000000000EEEEEEEE31
:1003D000EEEEEEEE00000000000000000000000065
:1003E000000000000000000000000000000000000D
:1003F00000000000000000000000000000000000FD
:1004000000000000000000000000000000000000EC
:1004100000000000000000000000000000000000DC
:10042000000000000000000000000000FFFFFFFFD0
:10043000FFFFFFFF000000000000000000000000C0
:1004400000000000000000000000000000000000AC
:10045000000000000000000000000000000000009C
:10046000000000000000000000000000000000008C
:10047000000000000000000000000000000000007C
:1004800000000000000DC0CC00000000000DD0D026
:1004900000000000CCCCCCCCCCCC0C0000B00000D8
:1004A000B0000D0000B00000B000CDCCCCB0C0CC8E
:1004B000B0C00C00D0B0000DB0000D00D0B0000DE9
:1004C000B0000D00D0B0000DB0C0DC00D0B0000D09
:1004D000B000D0CCCCB0C0CCB0C0CC00CCCCCCCC5C
:1004E000CCCCCCCC800008088800000008080808A4
:1004F0000808000008080808880000008808800034
:10050000080800000808800008080000000000003B
:10051000000000008800880808088000080808001B
:10052000880808080808880008080808080808005B
:1005300008080808880088080808800000000000F3
:10054000000000009000090999000000090909094C
:10055000090900000909090999000000990990009A
:1005600009090000090990000909000000000000C5
:100570000000000099009909090990000909090083
:1005800099090909090999000909090909090900CD
:10059000090909099900990909099000000000005A
:0405A0000000000057
:00000001FF
